:0A13250000010202030304040505A1
:1005E300E4F513F512F511F510C213C210C212C2CD
:1005F3001112078D7E0F7F008E418F4275490F7553
:100603004A12753F0F75401C75470F75483C754B73
:100613000F754C5CEE54E0700302072775140075E8
:1006230015808E168F17C374869FFF740F9ECF2479
:1006330002CF3400FEE48F0F8E0EF50DF50CF50B93
:10064300F50AF509F508AF0FAE0EAD0DAC0CAB0B0B
:10065300AA0AA909A808C31208D05026E515250B34
:10066300F582E514350AF58374CDF0E50B2401F525
:100673000BE4350AF50AE43509F509E43508F5080C
:1006830080C4E4F50BF50AF509F508AF0FAE0EAD1E
:100693000DAC0CAB0BAA0AA909A808C31208D050C9
:1006A30031AE0AAF0BE5172FF582E5163EF583E071
:1006B300FDE5152FF582E5143EF583EDF0EF2401FA
:1006C300F50BE43EF50AE43509F509E43508F508C8
:1006D30080B985144185154274002480FF740F345A
:1006E300FFFEC3E54A9FF54AE5499EF549C3E54444
:1006F3009FF544E5439EF543C3E5469FF546E5452F
:100703009EF545C3E5409FF540E53F9EF53FC3E5B4
:10071300489FF548E5479EF547C3E54C9FF54CE5F3
:100723004B9EF54BD2E843D82090E668E04409F0AD
:1007330090E65CE0443DF0D2AF90E680E020E10536
:10074300D2141210FD90E680E054F7F0538EF8C2F5
:10075300133011051203BFC211301329120BFE50BF
:1007630024C21312122B20101690E682E030E70405
:10077300E020E1EF90E682E030E604E020E0E412DE
:0A0783001159120EFE12141380C764
:1003BF0090E6B9E070030204701470030204ED2498
:1003CF00FE700302057024FB700302046A147003AD
:1003DF00020464146073146076240560030205CF71
:1003EF0012141640030205DB90E6BBE024FE6022E8
:1003FF0014603324FD601114602224067048E54117
:10040F0090E6B3F0E5428037E54990E6B3F0E54A70
:10041F00802DE54390E6B3F0E5448023E54590E673
:10042F00B3F0E546801990E6BAE0FF121185AA06EF
:10043F00A9077B01EA494B600DEE90E6B3F0EF9010
:10044F00E6B4F00205DB0205D41212F50205DB1249
:10045F0013960205DB1210510205DB1212E302059F
:10046F00DB12141840030205DB90E6B8E0247F602E
:10047F001514601924027063A210E43325E0FFA263
:10048F0012E4334F8041E490E740F0803F90E6BCA8
:10049F00E0547EFF7E00E0D394807C0040047D0119
:1004AF0080027D00EC4EFEED4F2425F58274133E45
:1004BF00F583E493FF3395E0FEEF24A1FFEE34E6DE
:1004CF008F82F583E0540190E740F0E4A3F090E6CB
:1004DF008AF090E68B7402F00205DB0205D4121449
:1004EF001A40030205DB90E6B8E024FE60162402F2
:1004FF0060030205DB90E6BAE0B40105C210020505
:10050F00DB0205D490E6BAE0705590E6BCE0547E6D
:10051F00FF7E00E0D394807C0040047D0180027D4B
:10052F0000EC4EFEED4F2425F58274133EF583E467
:10053F0093FF3395E0FEEF24A1FFEE34E68F82F5B3
:10054F0083E054FEF090E6BCE05480131313541F65
:10055F00FFE0540F2F90E683F0E04420F0806D8091
:10056F006412141C506690E6B8E024FE6019240251
:10057F00705A90E6BAE0B40104D210804F90E6BAF8
:10058F00E064026047803E90E6BCE0547EFF7E0050
:10059F00E0D394807C0040047D0180027D00EC4E0E
:1005AF00FEED4F2425F58274133EF583E493FF335C
:1005BF0095E0FEEF24A1FFEE34E68F82F5838008ED
:1005CF00120080500790E6A0E04401F090E6A0E012
:0305DF004480F065
:0105E20022F6
:030033000213FFB6
:0413FF0053D8EF329E
:100F00001201000200000040C01672290000010218
:100F100000010A0600020000004001000902200052
:100F200001010080320904000002FF0000000705F3
:100F300001024000000705820200020009022000B1
:100F400001010080320904000002FF0000000705D3
:100F5000010240000007058202400000040309046A
:100F60001003510048005900430061006D007300F8
:100F700016035100480059002D00380020002000C1
:080F80005600310030000000B2
:10095C00608018000104020202020207000000027B
:10096C00000002001332120A080C080000000000FC
:10097C000000003F01040202020202070000000214
:10098C000000020013320A12100C080000000000D4
:10099C000000003F033A03030A0A030700000002A9
:1009AC00000002001332120A080C080000000000BC
:1009BC000000003F033A03030A0A03070000000289
:1009CC000000020013320A12100C08000000000094
:1009DC000000003F602418870000000000000000A9
:1009EC0000000000000000000000000000000000FB
:1009FC00000000000000000000000000471880808C
:060A0C00000000CA4E00CC
:100AFC0090E60174CAF090E6F574FFF0901880E06F
:100B0C0090E6F3F0901881E090E6C3F0901882E044
:100B1C0090E6C1F0901883E090E6C2F0901885E062
:100B2C0090E6C0F0901886E090E6F4F075AF07748C
:100B3C0018F59A7400F59B759DE4E4F59EFF90E61C
:100B4C007BE090E67CF00FBF80F490E67174FFF0D0
:100B5C00F5B490E672E04480F043B680000000E407
:100B6C0090E6C4F000000090E6C5F0901887E09085
:100B7C00E6C6F0901888E090E6C7F0901889E090EF
:100B8C00E6C8F090188AE090E6C9F090188BE090D7
:100B9C00E6CAF090188CE090E6CBF090188DE090BF
:0B0BAC00E6CCF090188EE090E6CDF053
:010BB700221B
:03004300020C00AC
:03005300020C009C
:100C0000021273000212B9000212A30002128B003A
:100C1000020EC80002108E0002141E0002141F00F3
:100C20000214200002142100021422000212050006
:100C300002142300021424000214250002142600CA
:100C40000214270002141F000214280002142900B5
:100C500002142A0002142B0002142C0002142D008E
:100C600002142E0002141F0002141F0002141F00A1
:100C700002142F000214300002143100021432005A
:100C8000021433000214340002143500021436003A
:100C900002143700021438000214390002143A001A
:100CA00002143B0002143C0002143D0002143E00FA
:080CB00002143F000214400091
:1011590090E682E030E004E020E60B90E682E030A1
:10116900E119E030E71590E680E04401F07F147E54
:0C11790000120BB890E680E054FEF0225B
:10122B0090E682E044C0F090E681F0438701000035
:04123B00000000228D
:1010FD0030140990E680E0440AF0800790E680E025
:10110D004408F07FDC7E05120BB890E65D74FFF0AD
:0F111D0090E65FF05391EF90E680E054F7F022F8
:02118500A907B8
:10118700AE4BAF4C8F828E83A3E064037017AD0123
:1011970019ED7001228F828E83E07C002FFDEC3EDB
:0911A700FEAF0580DF7E007F0031
:0111B000221C
:100BB8008E1C8F1D90E600E054187012E51D24016C
:100BC800FFE4351CC313F51CEF13F51D801590E6E3
:100BD80000E05418FFBF100BE51D25E0F51DE51CCE
:100BE80033F51CE51D151DAE1C7002151C4E600565
:060BF80012123F80EE2204
:10123F007400F58690FDA57C05A3E582458370F9C2
:01124F00227C
:100A1200C106C18802240000023B00000237000028
:0C0A2200022B1040022E0000C107C1038F
:10078D0090E600E054E74410F000000000000090F7
:10079D00E61074A0F000000090E60B7401F090E6F6
:1007AD001274E0F0000000E490E613F000000090F9
:1007BD00E614F000000090E615F000000090E61839
:1007CD00740CF000000090E6D27402F090E6047410
:1007DD0080F00000007402F0000000E4F000000062
:1007ED00120AFCE490E671F075B4FF90E672F075B4
:1007FD00B6FF75B1FF90E670F075B2FFD2A212137D
:10080D0019D2A1752402752500C3E4952CFF74102F
:10081D00952BAD0790E630F0AF05EF90E631F0E4A3
:10082D00F53BF53CF537F53890E65EE04408F00011
:10083D000000E490E68DF053B0FD53B0FB53B0F7DC
:10084D0012101290E60174C8F043B00253B0FB537E
:10085D00B0F753B1F77FAA7E0012135753B1EF755E
:10086D0027007528B4753301753490752B10752CD0
:0A087D00B875350675362CE4F52D2C
:01088700224E
:03141300020CB810
:020BFE00D32200
:020EFE00D322FD
:02141600D322DF
:1010510090E680E030E71800000090E6207402F08E
:10106100000000E490E621F0000000D208801600A4
:101071000000E490E620F000000090E6217440F0CA
:0D108100000000C20890E6BAE0F532D3226C
:1012E30090E740E532F0E490E68AF090E68B04F074
:0212F300D32204
:0813960090E6BAE0F526D3222F
:1012F50090E740E526F0E490E68AF090E68B04F06E
:02130500D322F1
:02141800D322DD
:02141A00D322DB
:02141C00D322D9
:10008000E4F518F51990E6B9E01208E100ABB2000A
:10009000B2B300FAB4010CB502A3B602DAB702F6A5
:1000A000C10341C2038ED1000003BB90E74074B28C
:1000B000804DE490E68AF090E68BF090E6A0E02098
:1000C000E1F990E68BE0F518E4F53BF53CF5B5F584
:1000D000B390E60174CAF0E490E6C3F090E6C2F093
:1000E000D206D20400000090E6047480F000000004
:1000F0007402F0000000E40202EB90E74074B4F0F8
:10010000E490E68AF090E68B040202EBE490E68A43
:10011000F090E68BF090E6A0E020E1F990E68BE02D
:10012000F518D394174024E4F51974402519F58285
:10013000E434E7F583E0FF74AB2519F582E4341865
:10014000F583EFF00519E519B418DF90E6A0E04457
:1001500080F07F8A7E001213579018ABE0FF7E007C
:100160001213609018ABE0FF7E001213699018AB79
:10017000E0FF7E001213729018B2E075F004A4FF45
:10018000AEF012137B9018B2E075F004A4FFAEF04D
:100190001213849018B2E075F004A4FFAEF01213AD
:1001A0008D9018B0E0FF5480C4131313540124FF42
:1001B0009205EF5440C41313540324FF920CE054EF
:1001C00002C31324FF920D9018AFE0FF5480C413B4
:1001D0001313540124FF920BEF5440C41313540320
:1001E00024FF920FE0FF5408131313541F24FF92AF
:1001F00000EF54041313543F24FF9201E0FF540214
:10020000C31324FF920EEF13920AA20592A02000BE
:100210001090E6C0200B05744EF08013749CF080A3
:100220000E90E6C0200B05749FF08003749DF09043
:1002300018B1E0FF7004C209C202EFB40104C209A0
:10024000D202EFB40204D209C2029018B5E0FEA3B4
:10025000E07C002400F528EC3EF527A3E0FEA3E0B7
:100260002400F534EC3EF533A3E0FEA3E02400F5D2
:100270002CEC3EF52BA3E0FEA3E02400F536EC3E8B
:10028000F535A3E0FEA3E02400F531EC3EF530A304
:10029000E0F52DA3E0FEA3E02400F52AEC3EF529CD
:1002A0000203BDE4F51974AB2519F582E43418F5A1
:1002B00083E0FF74402519F582E434E7F583EFF01D
:1002C0000519E519B418DF000000E490E68AF00093
:1002D000000090E68B7418020384C20690E7407415
:1002E000B7F0E490E68AF090E68B04F090E6A0E0A8
:1002F0004480F00203BDE490E68AF090E68BF09033
:10030000E6A0E020E1F990E68BE0F518D3940240F6
:1003100024E4F51974402519F582E434E7F583E007
:10032000FF74C32519F582E43418F583EFF005193D
:10033000E519B403DF90E6A0E04480F0120FD3800B
:100340007C90E7407466F0A3741EF0A3740CF0A3D5
:100350007426F0A37407F0A374EEF0A37401F0E424
:10036000A3F0A37453F0300805E4A3F0800690E7EF
:100370004974FFF0000000E490E68AF0000000906D
:10038000E68B740AF090E6A0E04480F0802890E7C5
:100390004074CFF0000000E490E68AF00000009086
:1003A000E68B04F090E6A0E04480F012139E300C3F
:0E03B00002C2A21214431210128002D322C302
:0103BE00221C
:10127300C0E0C083C082D2115391EF90E65D740148
:08128300F0D082D083D0E032EC
:1012A300C0E0C083C0825391EF90E65D7404F0D038
:0612B30082D083D0E0327E
:1012B900C0E0C083C0825391EF90E65D7402F0D024
:0612C90082D083D0E03268
:100EC800C0E0C083C0828547438548448544828505
:100ED8004383A37402F0853F458540468546828555
:100EE8004583A37407F05391EF90E65D7410F0D03A
:060EF80082D083D0E0323D
:10128B00C0E0C083C082D2135391EF90E65D740827
:08129B00F0D082D083D0E032D4
:10108E00C0E0C083C08290E680E030E720853F4319
:10109E00854044854482854383A37402F085474589
:1010AE00854846854682854583A37407F05391EFA4
:0D10BE0090E65D7420F0D082D083D0E03247
:01141E00329B
:01141F00329A
:011420003299
:011421003298
:011422003297
:10120500C0E0C083C082C2AF75230000000090E635
:101215008DE4F05391EF90E65FE04408F0D2AFD053
:0612250082D083D0E0320C
:011423003296
:011424003295
:011425003294
:011426003293
:011427003292
:011428003291
:011429003290
:01142A00328F
:01142B00328E
:01142C00328D
:01142D00328C
:01142E00328B
:01142F00328A
:011430003289
:011431003288
:011432003287
:011433003286
:011434003285
:011435003284
:011436003283
:011437003282
:011438003281
:011439003280
:01143A00327F
:01143B00327E
:01143C00327D
:01143D00327C
:01143E00327B
:01143F00327A
:011440003279
:060A2F008F1A8C1B8D1CC8
:100A350075B6FF531A0753B1FE7F0A7E00120FBC2D
:100A4500E4F51DF51EC37402951EFFE51AA80708F7
:100A55008002C313D8FC30E00543B104800353B1D1
:100A6500FB7F0A7E00120FBC43B1027F0A7E001293
:100A75000FBC53B1FD7F0A7E00120FBC051EE51E9B
:100A85007002051DC39403E51D6480948040B6E49F
:100A9500F51DF51EC37409951EFFE51CAE1BA807C1
:100AA500088005CEC313CE13D8F930E00543B10451
:100AB500800353B1FB7F0A7E00120FBC43B1027F56
:100AC5000A7E00120FBC53B1FD7F0A7E00120FBCD7
:100AD500051EE51E7002051DC3940AE51D6480947C
:100AE5008040B143B1017F0A7E00120FBC53B1FEB5
:070AF5007F0A7E00020FBC26
:09135700AD07AC06E4FF020A2F09
:09136000AD07AC067F04020A2F60
:09136900AD07AC067F05020A2F56
:09137200AD07AC067F06020A2F4C
:09137B00AD07AC067F01020A2F48
:09138400AD07AC067F02020A2F3E
:09138D00AD07AC067F03020A2F34
:100F88007E00120FBC12130F7F147E00120FBC12CA
:100F980014037F037E00120FBC12140F7F027E0021
:100FA800120FBC1213397F027E00120FBC12134DB0
:040FB8007F027E0036
:100FBC00EF7803C333CE33CED8F9FFEF4E6007EF93
:070FCC001F70F81E80F522E2
:0713A6005380F75380DF22A2
:0713AD005380F7438020226A
:0713B4004380084380202262
:0713BB005380FE5380FB226A
:0713C2005380FE438004226A
:0713C9004380014380042270
:0414030053807F2271
:04140700438080227C
:04140B005380BF2229
:04140F0043804022B4
:0713D0005380F75380EF2268
:0713D7005380F74380102250
:0713DE004380084380102248
:0713E5005380FE5380FD223E
:0713EC005380FE4380022242
:0713F3004380014380022248
:0A12CF001213197F0A7E00120FBCF3
:0A12D9005380F75380DF5380EF22AB
:0A132F005380FE5380FB5380FD2223
:0A1339005380F74380204380102208
:081307007E00120FBC12133925
:0A130F005380FE4380044380022255
:0A13430043800843802043801022FD
:0A134D004380014380044380022224
:0C13190012133912140712134D02140BAA
:101250001212CF7F0312130712134312132F7F03AF
:10126000120F8812140B120FB81214077F147E008D
:03127000020FBCAE
:1011B1001212CF7F081213077F017E00120FBC129B
:1011C100134312132F7F02120F8812140B120FB840
:0A11D1001214077F147E00020FBC09
:1010CB0012131943B1087F017E00120FBC12130FCC
:1010DB00120FB8121343120FB81214037F02120F20
:1010EB009C12140B7F147E00120FBC12140743B119
:0210FB000822C9
:10112C00121319120FB8E4FFFE12130F121343120D
:10113C00140312140F12133912134D12140B121430
:0C114C00070FBF00010EBE03E0BFF7DD7F
:011158002274
:011441002288
:011442002287
:0513FA008E4D8F4E2214
:07139E00C2A1120FB8D2A199
:0113A5002225
:100FD300E4F5B375B5FF90E60174C8F0E4F51AF5CE
:100FE3001B43B0027F1E7E00120BB853B0FD7F1E61
:100FF3007E00120BB8051BE51B7002051AC394058E
:0E100300E51A6480948040D990E60174CAF02A
:0110110022BC
:10101200E4F5B375B5FF90E60174C8F0E4F51AF58E
:101022001B43B0047F0A7E00120BB853B0FB7F0A49
:101032007E00120BB8051BE51B7002051AC394054E
:0E104200E51A6480948040D990E60174CAF0EB
:01105000227D
:011443002286
:011444002285
:100D550043B00243B004121407121343200E0312CA
:100D6500139E300C02C2A21214439018ACE075F029
:100D750040A485F018F519AF237E00AC18AD191203
:100D85000888D3EF9400EE940040117F007E041292
:100D95000BB8E519151970DF151880DB9018ADE053
:100DA500751800F519AF237E00AC18AD1912088827
:100DB500D3EF9400EE940040117F007E01120BB832
:100DC500E519151970DF151880DB9018AEE0FF7E68
:100DD50000120BB8121444300C09D2A27FF47E0124
:090DE500120BB843B00253B0FB3D
:010DEE0022E2
:100E7B00EF4E7048752301300A0312112C200D051B
:100E8B00120D55800F121444300C09D2A27FF47E40
:100E9B0001120BB8200A06200E0312112C1212504D
:100EAB00E4FDFCC3ED9528EC9527500A1210CB0DF1
:0C0EBB00BD00010C80ED43B00253B0FB01
:010EC7002208
:1011DB00AB070000007F007C017D0012089A90E6AF
:1011EB00D0EFF0000000EB90E6D1F000000075BBF3
:0A11FB0004000000E5BB30E7FB2212
:100CB800200603020D54E5BB20E703020D5420046F
:100CC80003020D54AF3CAE3B120E7BD2A0000000D5
:100CD800E52B90E6D0F0000000E52C90E6D1F0007E
:100CE800000075BB04000000E5BB30E7FBE52D7094
:100CF800031210CBE52DB401061210CB1210CB0550
:100D08003CE53C7002053BC39536E53B9535403CD8
:100D1800C204AF31AE301211DBE4FDFCC3ED9534F3
:100D2800EC9533500A1210CB0DBD00010C80ED126A
:100D38001407121343E4F5B375B5FF90E60174C8C0
:0C0D4800F043B00253B0FB53B0F7C2A060
:010D5400227C
:03000000020DEFFF
:0C0DEF00787FE4F6D8FD75814E020E36C8
:10088800EF8DF0A4A8F0CF8CF0A428CE8DF0A42E84
:02089800FE223E
:10089A00C2D5EC30E709B2D5E4C39DFDE49CFCEE79
:1008AA0030E715B2D5E4C39FFFE49EFE120907C3E1
:1008BA00E49DFDE49CFC800312090730D507C3E4DC
:0608CA009FFFE49EFE22E8
:1008D000EB9FF5F0EA9E42F0E99D42F0E89C45F07E
:0108E00022F5
:1008E100D083D082F8E4937012740193700DA3A3A6
:1008F10093F8740193F5828883E4737402936860BA
:06090100EFA3A3A380DFB9
:100DFB000205E3E493A3F8E493A34003F68001F226
:100E0B0008DFF48029E493A3F85407240CC8C333F8
:100E1B00C4540F4420C8834004F456800146F6DFC7
:100E2B00E4800B010204081020408090095CE47EF2
:100E3B00019360BCA3FF543F30E509541FFEE493BC
:100E4B00A360010ECF54C025E060A840B8E493A383
:100E5B00FAE493A3F8E493A3C8C582C8CAC583CAAE
:100E6B00F0A3C8C582C8CAC583CADFE9DEE780BE66
:010A2E0000C7
:10090700BC000BBE0029EF8DF084FFADF022E4CCD4
:10091700F875F008EF2FFFEE33FEEC33FCEE9DEC9D
:10092700984005FCEE9DFE0FD5F0E9E4CEFD22EDE3
:10093700F8F5F0EE8420D21CFEADF075F008EF2F2D
:10094700FFED33FD4007985006D5F0F222C398FD1E
:050957000FD5F0EA22BB
:00000001FF
